:02000000C52F0A
:0A000600E80803190800F930FF3E76
:10001000031D0728E80B06280800FA30E800032033
:10002000FA30E8000320FA30E8000320FA30E80054
:100030000320CE0B0D2808008312031386158611AA
:1000400008000230831203130605E900EA010310D9
:10005000690CC5000800E908031930280615312885
:10006000061108006908EA0003106A0DE900023071
:100070006905E900FD300605EA0069086A048600A2
:100080000800630E0F3985001C20630885001C20C2
:100090000230E80003200800823083160313860034
:1000A00001308312E9002B2021204508E800E901F6
:1000B0002B200130E9003220803083168600831225
:1000C0006808C5000800ED01EC01EB01EA01EE0152
:1000D0006E1A82280310EA0DEB0DE40DE50DEC0D10
:1000E000ED0D67086D02031D772866086C02031C7E
:1000F00080286608EC026708031CED03ED026A1411
:10010000EE0A68286A08C5006B08C60008000610D9
:100110006108013A031991286108023A03199628E7
:10012000A0286208803EE3004120A028E501620883
:10013000403EE4000318E50A64088038E3004120EB
:100140000230E80003200800803083160313860085
:1001500001308312E9002B20E9013220E9012B2034
:10016000080083120313E9012B20E901322001303A
:10017000E9002B200130E90032200800E2010830BC
:10018000E300E4016408803A803C031DC928630849
:10019000003C0318E4286208E8000310680DE20040
:1001A000013061056204E2006108E800E901031022
:1001B000680CE1006408E500E3080319E503630344
:1001C000E3006508E400C2288030E300E40164082D
:1001D000803A803C031DEE286308003C031809297F
:1001E0006208E90032206208E800E9010310680CA7
:1001F000E2000130E9002B20E9012B206308E60032
:100200006408E7000310E70C660CE3006708E400ED
:10021000E7284C200800EE01ED01EC01EB01EF01B5
:100220006F1A2A290310EB0DEC0DE40DE50DED0D11
:10023000EE0D67086E02031D1F2966086D02031C80
:1002400028296608ED026708031CEE03EE026B1412
:10025000EF0A10296D08C5006E08C6000800C41812
:100260003329E301C4146008303EA5000430E300E4
:100270006308003C031892293D293E29DF1F5329BA
:100280005E09E4005F09E500E40A0319E50A0A30A3
:10029000E600E7010B214509E8004609E900E80A04
:1002A0000319E90A5F295E08E4005F08E5000A30E7
:1002B000E600E7010B214508E8004608E900680868
:1002C000303EEA00831320308400630884076A0804
:1002D00080006A296B29DF1F80295E09E4005F091D
:1002E000E500E40A0319E50A0A30E600E7016320A5
:1002F0004509E8004609E900E80A0319E90A8C29DA
:100300005E08E4005F08E5000A30E600E7016320CC
:100310004508E8004608E9006808DE006908DF00D3
:10032000E30338295E08303EA000E3016308053C82
:10033000031CB3296308620783169B00831283138F
:100340002030840063088407000883169A001C1577
:1003500055309D00AA309D009C149C18AD291C119D
:100360008312E30A9629080083120313D101823015
:100370008316860008308312D200D3015308803AD6
:10038000803C031DC5295208003C0318DF29510891
:10039000D5000310550DD1000130E9002B2021209C
:1003A00045085104D100E9012B205308D400D2089C
:1003B0000319D4035203D2005408D300BE290130DC
:1003C000E90032205108C5000800680883169B0028
:1003D0001C141A088312C50008005E08E1005F08BB
:1003E000E200872006146008E30041200800DD01D8
:1003F0005D08053C031C5D2A5708E1005D08053CCB
:100400005807E200872006145D08033A031D0D2AF1
:100410002E30E3004120DD0A5C2A0E2A0F2ADA1F63
:10042000242A5909E4005A09E500E40A0319E50AF7
:100430000A30E600E7010B214509DE004609DF002E
:10044000DE0A0319DF0A302A5908E4005A08E500D9
:100450000A30E600E7010B214508DE004608DF0010
:100460005E08303EE3004120352A362ADA1F4B2A47
:100470005909E4005A09E500E40A0319E50A0A30BB
:10048000E600E70163204509E2004609E300E20ACD
:100490000319E30A572A5908E4005A08E5000A300C
:1004A000E600E70163204508E2004608E300620831
:1004B000D9006308DA00DD0AF8295708E1005D0871
:1004C0005807E000DD0A6008E200872006142C309F
:1004D000E30041205708E1005D085807E000DD0A0D
:1004E0006008E20087200614752A762ADC1F8B2A12
:1004F0005B09E4005C09E500E40A0319E50A0A3037
:10050000E600E7010B214509DE004609DF00DE0AAF
:100510000319DF0A972A5B08E4005C08E5000A304B
:10052000E600E7010B214508DE004608DF005E0813
:10053000303EE3004120DD010800441BA42ADD0118
:10054000DE01DF01E0014417DC01DB0104305B0266
:100550005C080318AD2A0319AF2ADC1FB02AB12AA0
:10056000E72AB22AB32AD81FC42A5709E400580937
:10057000E500E40A0319E50A1030E600E7010B2163
:100580004509E800E80ACE2A5708E4005808E500C3
:100590001030E600E7010B214508E80083135D30C9
:1005A00084005B08840768088000570EE1000F3064
:1005B000E105580EE200F039E1040F30E205610870
:1005C000D7006208D800DB0A0319DC0AA62AA42097
:1005D0005A08E100BE205F0EF039E200620E0F39CA
:1005E000E300600EF0396307E100BE205D0EF039D4
:1005F000E200620E0F39E3005E0EF0396307E1009E
:10060000BE20CE30E100BE205908E100BE20B1205E
:10061000F03083168500F03086000800EA01EC0116
:10062000EB015208ED005308EE00EA19252B511C8E
:100630001F2B6D08EB070318EC0A6E08EC07D10CB2
:100640000310ED0DEE0DEA0A152B6B08C5006C08C2
:10065000C6000800EA01EC01EB015A08ED00EE01CA
:10066000EA19402B5B1C3A2B6D08EB070318EC0AC8
:100670006E08EC07DB0C0310ED0DEE0DEA0A302BD3
:100680006B08C5006C08C60008008312031306102F
:100690000130E30041200230E8000320080083120B
:1006A0000313861106100530E8000320033085008F
:1006B0001C200530E8000320023085001C20053096
:1006C000E80003202830E30041200130E800032047
:1006D0000830E30041200130E80003200C30E30043
:1006E00041200130E80003200630E30041200800EB
:1006F000A4204F08E100BE20B4214508D000B1205D
:10070000F03083168500F030860083125008C50053
:10071000080044188D2BCF0144144F08053C031CDE
:100720009E2B4F084E07E800E521831320308400FC
:100730004F08840745088000CF0A8D2BCF01250E76
:10074000F039E800E9010310E80C0310E80C03108D
:10075000E80C0310680CB0006908B100200EF039F5
:10076000D000500E0F39D1001030D2002730D30006
:100770000E234508D7004608D800210EF039D400D2
:10078000540E0F39D100E830D2000330D3000E23CD
:100790004508D5004608D60055085707DE0056081C
:1007A000DF0058080318DF0ADF07220EF039D900EE
:1007B000590E0F39DA006430DB002A234508DC00CB
:1007C0004608DD005C085E07E3005D08E4005F08A2
:1007D0000318E40AE407230EF039E000600E0F3935
:1007E000DA000A30DB002A234508E1004608E2006F
:1007F00061086307E6006208E70064080318E70A77
:10080000E707240EF039E500650E0F396607E800AA
:100810006708E9000318E90A6808C5006908C60006
:100820000800C419162CD201D101C415441A1C2C7D
:100830000130D300D4014416C41A212CD601D501AD
:10084000C4164208DE000B30DF007F30E000ED21EF
:1008500032082E02DB00330A031833082F02DC00B3
:1008600038085B07DD003908DE005C080318DE0A83
:10087000DE075D08DF005E08E0000310DF0DE00D1D
:100880000310DF0DE00D0310DF0DE00D30085F07F2
:10089000E1003108E20060080318E20AE20761089B
:1008A000D7006208D8004308D9004F08DA009D221B
:1008B00001308312360603193708031D642C3208F1
:1008C000D1003308D200682C2E08D1002F08D200A6
:1008D0004208D7000330D8005108D9005208DA0086
:1008E0003008DB003108DC00F7215108DE00520837
:1008F000DF003008E0003108E1005008E2002F215D
:100900000A30E8000320D308031D892CD4080319FA
:10091000A12D060E0F390E3A031D9B2C4208DE0056
:100920000B30DF002030E000ED21B701B6010130CF
:10093000D300D4010800060E0F39073A031D0B2D12
:100940004208DE000230DF007E30E000ED21420888
:10095000023A031DC02CBE08031DB92CBF08031D9D
:10096000B92CD830AE000430AF000130BE00BF015A
:10097000BF2CFC30AE000830AF00BF01BE01FF2C21
:10098000B608031DF62CB708031DF62CC008031D7E
:10099000DA2CC108031DDA2CF630AE002830AF0087
:1009A0003408B2003508B300F030C3000130C00095
:1009B000C101F62C0130400603194108031DEC2C3F
:1009C000FC30AE000830AF00B301B201F030C3001C
:1009D0000230C000C101F62CD830AE000430AF00A8
:1009E000B301B201F030C300C101C0012E08DE0026
:1009F0002F08DF00E101E0015008E2002F21C8309C
:100A0000E80003204208DE000230DF002030E00072
:100A1000ED21D401D30180300505D700DA01003083
:100A200057020319DA0A060E0F39D800D9010D3022
:100A300058020319D90A59085A04DD00060E0F3965
:100A4000DB00DC010B305B020319DC0A5C085D048F
:100A50000319A02D40300505DE00E10100305E02E3
:100A60000319E10A060E0F39DF00E0010D305F02C5
:100A70000319E00A6008610403196B2DBA08031D0D
:100A8000442DBB0803195C2D0130360603193708C5
:100A9000031D4E2DB20A0319B30A5B2D3C082E0725
:100AA000E2003D08E3002F080318E30AE3076208A9
:100AB000AE006308AF006A2DB00A0319B10A0A300C
:100AC000300603193108031D6A2DAE0A0319AF0A57
:100AD000B101B0019E2DBA08031D712DBB08031989
:100AE000892D0130360603193708031D7C2DB20805
:100AF0000319B303B203882D3C082E02E2003D0A1D
:100B000003183D082F02E3006208AE006308AF003F
:100B10009E2DB0080319B103B0030030FF30310639
:100B2000031D9E2D3008FF3A031D9E2DAE08031DA8
:100B30009A2DAF03AE030930B000B101D401D30147
:100B4000832C0130D300D40132082E02D700330A9F
:100B5000031833082F02D8005708D5005808D600CC
:100B60000B305602031DB62DB9305502031CD42D8F
:100B7000D61BD42DB208031DC02DB3080319CE2DEA
:100B80003208523ED7003308D80003300318D80A81
:100B9000D8075708AE005808AF00D22D5230AE002B
:100BA0000330AF00B101B0015608033C031DDA2D3C
:100BB0005508513C0318DE2DD61FF82DB208031D31
:100BC000E42DB3080319F22D3208B83ED7003308DC
:100BD000D8000B300318D80AD8075708AE005808B9
:100BE000AF00F62DB830AE000B30AF00B101B00150
:100BF000282CD10151080F3C031C0E2E4F08E10098
:100C00005108E2008720061451085007E800E5214A
:100C100037304502E3004120D10AFA2DD101080006
:100C200083120313CA01C9010130CB00CC01063085
:100C3000CD00F03083168500F03086004030810012
:100C400083128B014F236830CE0089234508A6000C
:100C50004608A7003008A8003108A9007030CE006F
:100C600089234508AA004608AB003008AC003108CB
:100C7000AD007830CE0089234508B2004608B300A5
:100C80003208B4003308B5000130CF004030D00046
:100C9000F9250230CF005030D000F9250230CE00C7
:100CA0000D20CB08031D572ECC0803197C2E0130D4
:100CB000CF00D001F9250230CF001030D000F92547
:100CC0000130D7000330D8002608D9002708DA0001
:100CD0002808DB002908DC00F7210230D7000330A8
:100CE000D8002A08D9002B08DA002C08DB002D08D0
:100CF000DC00F721CC01CB0132082602D300330AF5
:100D0000031833082702D40038085307D5003908E0
:100D1000D60054080318D60AD6075508DB00560833
:100D2000DC000310DB0DDC0D0310DB0DDC0D03100C
:100D3000DB0DDC0D28085B07DD002908DE005C0800
:100D40000318DE0ADE075D08D7005E08D8004308F6
:100D5000D900C630DA009D2283122A08D3002B085E
:100D6000D4000310D30DD40D0310D30DD40D0310F4
:100D7000D30DD40D2C085307D5002D08D6005408E8
:100D80000318D60AD6075508D7005608D800F03001
:100D9000D900C030DA009D22C7308312CF007823FB
:100DA0004508C8004808FF3A031DD92E3F30C70048
:100DB000E02E481FDE2E2A30C700E02E2130C7006B
:100DC0000130DE000C30DF004708E000ED21C130CB
:100DD000CF0078234508C8004808FF3A031DF32ECA
:100DE0003F30C700002F481FFB2E831605122A3004
:100DF0008312C700002F8316051621308312C70007
:100E00000230DE000C30DF004708E000ED21060E66
:100E10000F39CE004E08073A03191F2F4E080B3A20
:100E20000319542F4E080C3A03197F2F4E080D3A20
:100E30000319A72F4E080E3A0319C12FC12F4523BE
:100E40000130CF002030D000F925BA08031D342F1F
:100E5000BB08031D342F0130BC00BD010630CD009E
:100E60000130BA00BB01462F01303A0603193B0896
:100E7000031D432F0A30BC00BD010A30CD000230F3
:100E8000BA00BB01462FCD01BB01BA010130DE0023
:100E90004D08DF002330E000ED21FA30E8000320A8
:100EA0000130CB00CC01C12F2A08AE002B08AF00C7
:100EB0002C08B0002D08B1000230C2003208C90071
:100EC0003308CA00B301B201B901B801C030CF0084
:100ED0007030D00011242E08AA002F08AB00300873
:100EE000AC003108AD004908B2004A08B300E03058
:100EF000B8000130B9000130CB00CC01C12F270868
:100F0000273C031D852F2608103C0318A62FA71B7E
:100F1000A62F45230130CF003030D000F925260818
:100F2000AE002708AF00B101B0010130B600B70133
:100F30000130C2000130BA00BB01C630CF007830AA
:100F4000D00011240130CB00CC014523C12F26084D
:100F5000AE002708AF002808B0002908B100013012
:100F6000C200C630CF006830D00011242E08A60081
:100F70002F08A7003008A8003108A9000130CB00D5
:100F8000CC013230E8000320512E831203134410A9
:100F9000C4104411C4114412C4124413F630A60004
:100FA0002830A700A901A801A030AA000230AB0098
:100FB000AD01AC01AF01AE01B101B001B830B2007A
:100FC0002430B300B501B401B701B601E030B80078
:100FD0000130B9000130BA00BB010130BC00BD01D5
:100FE0000130BE00BF010130C000C1010130C200AC
:060FF000F030C300102EDA
:02400E0050025E
:104200008900AF004B004B004B004B004B004B00B4
:104210004B004B004B004B004B0084007F00B10073
:104220008B00AF004B004B004B004B004B004B0092
:104230004B004B004B004B004B0084007F00B10053
:104240004B0067006500680084004B004B0068006D
:1042500084004B004B006800670084007F00B100C1
:10426000860083004B004B004B004B004B004B0083
:104270004B004B004B004B004B0084007F00B10013
:1042800080008E00690083007D007B004B00780079
:104290008B008D004B00640089008B008F00640050
:1042A0008A008E004B0089009C00A30065004B0033
:1042B0006900650069004B006900670067006C00D9
:1042C0002D002D002D002D002D002D002D002D0086
:1042D000310030003400380036003000FF00FF00AD
:1042E000300031003200340030003000FF00FF00A9
:1042F000300039003400300030003000FF00FF0093
:00000001FF
